:020000040800F2
:10000000000800203D3C0008A10C0008A30C0008DB
:1000100000000000000000000000000000000000E0
:10002000000000000000000000000000A50C000817
:100030000000000000000000A70C0008A90C000848
:10004000BD3C0008BD3C0008BD3C0008BD3C0008AC
:10005000BD3C0008BD3C0008BD3C0008BD3C00089C
:1000600000000000BD3C0008BD3C0008BD3C00088D
:10007000BD3C0008BD3C000800000000BD3C00087D
:100080000000000000000000000000000000000070
:10009000BD3C00080000000000000000B10C00089A
:1000A00000000000BD3C000800000000000000004F
:1000B000BD3C0008BD3C000800000000000000003E
:1000C00010B5064C2378002B07D1054B002B02D02E
:1000D000044800E000BF0123237010BD1800002079
:1000E000000000002C3D0008044B10B5002B03D08D
:1000F0000349044800E000BF10BDC04600000000F6
:100100001C0000202C3D000802B47146490849003B
:10011000095649008E4402BC7047C04602B471467D
:1001200049084900095C49008E4402BC7047C0463A
:10013000002243088B4274D303098B425FD3030A26
:100140008B4244D3030B8B4228D3030C8B420DD339
:10015000FF22090212BA030C8B4202D312120902C7
:1001600065D0030B8B4219D300E0090AC30B8B4205
:1001700001D3CB03C01A5241830B8B4201D38B03B3
:10018000C01A5241430B8B4201D34B03C01A524158
:10019000030B8B4201D30B03C01A5241C30A8B429B
:1001A00001D3CB02C01A5241830A8B4201D38B0286
:1001B000C01A5241430A8B4201D34B02C01A52412A
:1001C000030A8B4201D30B02C01A5241CDD2C3099C
:1001D0008B4201D3CB01C01A524183098B4201D318
:1001E0008B01C01A524143098B4201D34B01C01A03
:1001F000524103098B4201D30B01C01A5241C3087B
:100200008B4201D3CB00C01A524183088B4201D3E9
:100210008B00C01A524143088B4201D34B00C01AD5
:100220005241411A00D20146524110467047FFE741
:1002300001B5002000F006F802BDC0460029F7D045
:1002400076E770477047C046002B11D1002A0FD1C6
:10025000002900D1002802D00021C943081C07B49E
:10026000024802A14018029003BDC046D9FFFFFF1B
:1002700003B4684601B5029800F006F8019B9E465B
:1002800002B00CBC7047C046F0B557464E464546D6
:10029000DE46E0B504000D009246994683B08B42DD
:1002A00030D82DD04946504600F0BAF82900060053
:1002B000200000F0B5F8331A9846203B9B4633D413
:1002C0005A465346934042461F00534693401E00F1
:1002D000AF423AD8AF4200D178E05B46A41BBD41A3
:1002E000002B00DA75E00022002300920193012325
:1002F0005A4693400193012342469340009328E0DD
:100300008242CFD900220023009201930C9B002B44
:1003100001D01C605D600098019903B03CBC904620
:100320009946A246AB46F0BD424620239B1A524650
:10033000DA40414613004A468A40170042461F43AE
:10034000534693401E00AF42C4D9002200230092BE
:1003500001934346002BD9D0FB0772081A43464647
:100360007B080EE0AB4201D1A2420CD8A41A9D41F9
:10037000012024196D410021013E24184D41002E19
:1003800006D0AB42EED9013E24196D41002EF8D1C2
:10039000009801995B4600196941002B24DB2B0072
:1003A0005A464446D3402A00E2401C005B461500F2
:1003B000002B2ADB26009E40330026004746BE4025
:1003C0003200801A9941009001919FE7A342BCD866
:1003D00083E74246202300219B1A002200910192CC
:1003E0000122DA40019286E7424620239B1A2A0026
:1003F00046469A402300F340444613432A00E24015
:100400001C005B461500002BD4DA42462F00202347
:10041000260097409B1ADE403B003343CDE7C046A1
:1004200010B5002903D100F007F8203002E0081CC5
:1004300000F002F810BDC0461C2101231B049842A5
:1004400001D3000C10391B0A984201D3000A083965
:100450001B09984201D30009043902A2105C40181C
:100460007047C046040302020101010100000000C0
:1004700000000000F0B585B000F050F9FA2040000F
:1004800001F092FD694C0221694A200003F0B0F9A5
:10049000684B0221684A00932000684B03F0A8F9DA
:1004A00000F0CEFA00F0D8FA002800D1A0E0644DA8
:1004B000644E2800310000F0A3FA2B681B78013B42
:1004C000032B00D98CE06B460027280031005F73B6
:1004D0009F73DF7300F094FA0F236B4431780D2281
:1004E00000930E2328686B446A4403F07DFB564D4D
:1004F000B84270D002212000544A03F079F96B46CB
:10050000587B0138032863D80223514EFFF706FEBB
:1005100002323F50737000230122B3700433F37032
:10052000503373710C3BB371043332703271F37119
:10053000484A443B2B700221200003F059F92B78E4
:10054000082B4BD90A232B7001F028FD424B297848
:10055000C6183F4800F08CFA00F07EFA00283FD120
:1005600001F01CFD8642F7D2042120003B4A03F033
:100570003FF935E00022711D301D33707370B27089
:10058000F37000F057F90623354A2B70D3E77370E8
:1005900000230322B37004333270F370B21DF31DD5
:1005A000711D301D00F056F908232E4A2B70C2E74A
:1005B0000422737000233270B370F270F31DB21D09
:1005C000711D301D00F05EF90823274A2B70B2E739
:1005D000264A2F70AFE7264A2870ACE7002BB3D12C
:1005E00000F024FA00F038FA0028FBD000F028FAD6
:1005F00001F0D4FC1F4D2B68984206D300F0E0F8C0
:1006000001F0CCFCF530FF30286001F0C7FC1A4D3A
:100610002B68984200D245E700F0ECF801F0BEFCF0
:10062000FA239B00C01828603CE7C046583D0008EC
:10063000473D00087B3D0008693D00085D3D00081E
:10064000400000203400002035000020843D0008D8
:10065000000000208C3D000888130000993D000830
:100660008E3D0008903D0008923D0008943D000832
:10067000963D00083C0000203800002010B598B0DE
:10068000202200210CA803F048FB14220021684618
:1006900003F043FB1822002105A803F03EFB1D498F
:1006A0001D4A0B6801241A4080231B0113430B6071
:1006B00002230B931493002315938023DB021693DC
:1006C00080231022DB030BA80E940F92179301F0E6
:1006D000BDFC002800D0FEE70F230290009303909A
:1006E0000C3B049021006846019301F0FBFE0028BA
:1006F00000D0FEE70A230593063B0793802305A855
:100700005B01099301F0CCFF002800D0FEE718B090
:1007100010BDC04600700040FFE7FFFF10B501F0BC
:100720001DFCFFF7ABFF00F0C5F800F009FB00F07F
:10073000FBF900F055FA00F0F5F800F0B1FB0123E9
:10074000064C2268200011680B43136002F010FA77
:100750000021200002F03AFA10BDC046FC00002043
:10076000FEE70000F0B5022500260400134F85B017
:100770002A00019102A8390003F0C6FA02AB5B1906
:100780002A00390003A81E7003F0BEFA02AB02A9CA
:10079000012290209E7100F05AFC2A0003A99020AB
:1007A00000F072FC02AB1B79237002AB5A7905236F
:1007B000D2095343019A137005B0F0BD443D0008BF
:1007C00010B507490748FFF7CDFF012000F026FBD1
:1007D000054B1860054800F021FB054B186010BD63
:1007E0004D0000204C0000204800002000020024A2
:1007F000440000201FB5094A094B12681B78029279
:10080000084A022112685BB20192074A074812782F
:100810000092074A02F0ECFF05B000BD4400002042
:100820004C000020480000204D000020BD3D000885
:10083000A43D0008002807D0002905D0034B1B78F1
:100840000370034B1B780B707047C0464C000020B0
:100850004D00002030B5002811D000290FD0002A0B
:100860000DD0002B0BD0064C25681D7023681B0A89
:10087000137023681B0C0B7023681B0E037030BDB4
:100880004800002030B5002811D000290FD0002AE0
:100890000DD0002B0BD0064C25681D7023681B0A59
:1008A000137023681B0C0B7023681B0E037030BD84
:1008B0004400002030B5012489B01422002103A88F
:1008C00003F02BFA0221154BDA6A2243DA62DA6A64
:1008D00022400192019ADA6A0A43DA62DB6A0B402B
:1008E0000293029BBFF34F8F0D4D0022280006316B
:1008F00002F040F8082304940024280003A903937D
:100900000594069401F088FF4023280003A903936F
:100910000494059401F080FF09B030BD001002403E
:100920000004005010B50F4B0F4CFF2223600F4BFB
:10093000200063602623A360253BE360002323613E
:10094000A361E36180239B026261236200F002FDE8
:10095000002801D0FFF704FF0021200001F0B4FAC5
:1009600010BDC04600540040B0000020382960206F
:10097000082330B58FB00893802308A85B010C933F
:1009800001F08EFE02221B4BA025D96A01241143DF
:10099000D962D96AED05114001910199D96A2800FF
:1009A0001143D962D96A0A400292029A8022996B55
:1009B00092030A439A6380239B000393EF3BFF3B20
:1009C000049303A90F3B06930594079401F024FFB9
:1009D00080232800DB0003A90393079401F01CFF88
:1009E00022000021172001F0F5FF172002F01CF86B
:1009F0000FB030BD0010024010B501F063FA10BD19
:100A000010B5002801D0002905D10421044A054869
:100A100002F0EEFE10BD044B03601E230B70F9E7DD
:100A2000C23D0008D43D00084E00002000231900FC
:100A3000024AD15401331E2BFBD170474E000020D7
:100A400010B51E220249034800F082FD10BDC046C9
:100A50004E000020B000002010B5044801F02EFA2E
:100A6000203843425841C0B210BDC046B0000020FB
:100A700010B50B4A002802D01D2906D9094A0421C5
:100A8000094802F0B5FE002010BD8AB2074B0100F4
:100A9000074800F0B5FC44426041C0B2F4E7C046EC
:100AA000D83D0008E93D0008D43D0008FFFF0F00D5
:100AB000B000002080230268DB059A4206D10123A2
:100AC000034A916B0B439363BFF34F8F7047C0464C
:100AD0000010024010B5040086B01422002101A8C5
:100AE00003F01BF980232268DB059A4217D101200D
:100AF0000C4AD16A0143D162D36A01A90340009331
:100B0000009B202301931E3B02930023A02003930C
:100B100003330493C0050233059301F07DFE06B054
:100B200010BDC0460010024010B58AB0102200214E
:100B300002A803F0F2F808220021684603F0EDF85D
:100B40001022002106A803F0E8F88023234CDB05DF
:100B50000A222360002320006360A360E260236117
:100B6000636101F0EAFF002801D0FFF7F9FD80235F
:100B700020005B0102A9029302F096F8002801D040
:100B8000FFF7EEFD200002F006F8002801D0FFF785
:100B9000E7FD0023694620000093019302F024F949
:100BA000002801D0FFF7DCFD30230022069320004F
:100BB0002B3B06A907930892099202F019F8002826
:100BC00001D0FFF7CDFD08232268200091690B4377
:100BD0009361FFF77FFF0AB010BDC046FC00002004
:100BE0000B480C4B10B50360E1235B020C22436001
:100BF000002342618360C36003618361C361036258
:100C0000436202F069FB002801D0FFF7A9FD10BD87
:100C1000380100200044004010B5040086B01422C2
:100C2000002101A803F079F8124B22689A421ED1E4
:100C30008022114B9202996B0A4301219A63DA6A6E
:100C40000A43DA62DB6A0B400093009BBFF34F8FCD
:100C50000A4BA02001930223029300230393033342
:100C60000493C0055B1801A9059301F0D5FD06B0FA
:100C700010BDC04600440040001002400480000047
:100C800010B58AB2024B0100024802F087FA10BD8B
:100C9000FFFFFF013801002010B5FFF7F1FF10BD85
:100CA0007047FEE77047704710B501F06BF910BD53
:100CB00010B5044C200001F0C1F8200000F076FCD3
:100CC00010BDC046B00000200122054B596B0A43FD
:100CD0005A638022996B52050A439A637047C04653
:100CE000001002408022104B520019680A431A601B
:100CF000DA680E490A40DA601A680D490A40012193
:100D00001A609A688A439A601A680A490A401A6007
:100D1000DA6809490A40DA6000221A618022074B2A
:100D200012059A607047C046001002400C40FF88D0
:100D3000F6FFF6FEFFFFFBFFFFFF02FF00ED00E006
:100D4000072210B5154C0023A263C222FF32626253
:100D500022002C321370124A20002260902292034B
:100D600062600122238422610332E363A36223636E
:100D70006363A360E3606261A361E36102F02CFB43
:100D8000002801D0FFF7ECFC0021200002F0E0FC7D
:100D9000002801D0FFF7E4FC10BDC046B8010020D8
:100DA0000024014070B5040088B01422002103A87B
:100DB00002F0B3FF164B22689A4226D18022154BCF
:100DC0009200596B02240A435A630122A020032691
:100DD0000025D96AC0051143D962D96A1140019131
:100DE0000199D96A2143D962DB6A03A9234002939E
:100DF000029B03920496059501F00EFD064803A997
:100E000003940496059501F007FD08B070BDC04637
:100E1000002401400010024000040050802313B55C
:100E2000094C5B01694600902000019302F03CFCF4
:100E3000200002F0ABFB01212000494202F0D2FB6E
:100E4000200002F02DFC16BDB801002010B51021C5
:100E5000034801F089FD013843425841C0B210BD3A
:100E60000004005010B52021034801F07DFD013839
:100E700043425841C0B210BD0004005010B501F00B
:100E8000E9FB06490524FFF753F944432300013CDD
:100E9000002B00D110BDC046C046F7E740420F000E
:100EA00030B5144C87B01422002101A802F035FFA0
:100EB00020000122102101F05DFD012220002021EF
:100EC00001F058FD3023012501931F3B20000293C0
:100ED00001A90E3B0493039501F09EFC2A0020001B
:100EE000202101F047FD2A001021200001F042FDE1
:100EF00007B030BD0004005010B5134C2378002B10
:100F000011D001222021114801F034FDFFF7B6FF76
:100F1000012210210D4801F02DFDFFF797FF002859
:100F2000FBD0FFF7ABFFFFF79DFF00222021074812
:100F300001F020FDFFF7A2FF00221021034801F07D
:100F400019FD0123237010BD6C0000200004005027
:100F5000002220210E4810B501F00CFDFFF78EFF96
:100F6000012210210A4801F005FDFFF76FFF00285C
:100F7000FBD0FFF783FF01222021054801F0FAFC96
:100F8000FFF77CFFFFF76EFF0022024B1A7010BDC7
:100F9000000400506C00002010B50122041E00D196
:100FA000020020210C4801F0E5FCFFF767FF012259
:100FB0001021094801F0DEFCFFF760FFFFF746FF54
:100FC0000028FBD0002C01D0FFF74CFF002210219D
:100FD000014801F0CFFC10BD000400500122202187
:100FE0000D4810B501F0C6FCFFF748FF01221021A3
:100FF000094801F0BFFCFFF729FF0028FBD0FFF7ED
:101000003DFFFFF72FFF040000221021024801F0EE
:10101000B1FC200010BDC0460004005070B50D00AA
:101020001400002801D0FFF767FF0826E009013E01
:101030006400FFF7B1FFE4B2002EF7D1FFF7CEFF57
:101040000400002D01D0FFF783FF200070BD70B5B4
:101050000C001600002102000120FFF7DFFF002531
:10106000731E9D4208DBA419013C01212278002057
:10107000FFF7D4FF012070BD0021625D080001353B
:10108000FFF7CCFFEDB2EBE7F7B5012301920200C9
:101090000F00180000211A43FFF7C0FF0025019B35
:1010A000591E8D4213DB082500247F18FFF796FF99
:1010B0006400013D0443EDB2E4B2002DF6D10120FD
:1010C000FFF76AFFFFF744FF01203C70FEBD0826D2
:1010D00000247B190093FFF781FF6400013E044365
:1010E000F6B2E4B2002EF6D13000FFF755FF009BB8
:1010F00001351C70EDB2D2E703689A69920701D5F9
:1011000000229A6201229969114202D199690A4327
:101110009A61704730B5039C1204006822431A4359
:10112000054B45688905640D890D1C43A5430A4399
:101130002A43426030BDC046FF63FF0310B5436BD6
:10114000144C0AB2A34202D0134CA3420ED1002A7F
:101150000ADB9023102917D0303B202914D000231C
:10116000402911D10B430FE0B823F9E700239A423D
:1011700000DAB833CA0701D5F22213438A0701D532
:10118000F42213432029EDD001680A6813430B6051
:1011900010BDC0461D1D0008111C0008002310B51D
:1011A000CA0708D5030041331A7828231A401A3396
:1011B000282A00D0B0338A0708D5020028244132FB
:1011C00012782240A2420BD14422134309B20029D3
:1011D00001DAB822134301680A689A430A6010BD15
:1011E000F422F2E7F8B5036816009A6904001023A8
:1011F00010000D00202718401A4218D1F8BD6A1CB3
:1012000016D000F0CBFE801BA84201D8002D0ED1D5
:101210002022636C13436364230041331A7022005D
:10122000002342324034137001202370E6E7236824
:101230009A693A42E3D010222000DA61DF61FFF7B9
:101240005BFF2268054953680B4053600423626CBE
:1012500013436364230041331F70E0E700E800FE9E
:10126000F8B504000D001600202723689B693B4257
:1012700001D00020F8BD320029002000FFF7B2FFA6
:10128000002813D100F08AFE801BA84201D8002D4F
:10129000EBD12022636C13436364230041331A7043
:1012A0002200002342324034137023700120E1E712
:1012B000F8B504000E0017001D0022689369334042
:1012C0009B1B59424B41BB4201D0002017E06B1CD5
:1012D000F4D000F063FE069BC01AA84201D8002D8E
:1012E000EBD12022636C012013436364230041335C
:1012F0001A70220000234232403413702370F8BD6C
:10130000F8B504000D001600022723689B693B42D4
:1013100001D00020F8BD320029002000FFF762FF55
:10132000002815D16B1CF0D000F038FE801BA842BD
:1013300001D8002DE9D12022636C1343636423009C
:1013400041331A702200002342324034137023705C
:101350000120DFE770B504000120002C3FD02500FC
:1013600041352B78DAB2002B05D123004033200021
:101370001A70FFF7FDFA242301212B702368E0681F
:101380001A68A6688A431A6061681A4A0A401A6194
:101390009968194A11409960012821D180210902D8
:1013A000314399605868154901435960D968002054
:1013B0000A40DA60616922690A43A16909020A43A5
:1013C000DA60216AE2690A431A60012219680A4355
:1013D0001A60202360642B7020634234207070BD3B
:1013E00084210902314399600228DBD1802109015F
:1013F0005960D7E7FFFFFFF0FF7FFFFF008000028B
:10140000F0B51D00030087B04133049103931B78AE
:101410001600DAB2040005920220202B07D1002921
:1014200001D0002E05D180239B006364012007B00A
:10143000F0BD230040331A780220012AF7D00122A0
:101440001A7000F0ABFD2123039A070013702300EC
:10145000059A42331A7000222168049B62646685F3
:1014600063623A484B68626303404B6020002B0084
:1014700008210097FFF71CFF2368021E05D0802279
:10148000596812020A435A60D0E70826DE61E36811
:10149000022B09D12B00310020000097FFF708FF35
:1014A00023680028EBD1DE6180212B000022200080
:1014B00000974902FFF7FCFE002814D02268802321
:1014C00051681B020B435360B0E7FFF719FF226816
:1014D0000028F4D1636A1978013391626362638DE5
:1014E000013B9BB26385638D3A00290020009EB2C8
:1014F000002BEAD1FFF7B4FE236800280AD080222F
:10150000596812020A435A60626C0120042A00D012
:101510008DE76664802620223602DA6131002B00D6
:101520001F3A20000097FFF7C3FE23685A6816434E
:101530005E60002800D079E72022039B1A70230008
:10154000403442331870207071E7C046FF7FFFFFC0
:10155000F8B5030041331D780224EEB2202D1AD1D4
:10156000050040352F78012F15D020341C70002441
:101570005E70066844647368084F3B407360428540
:10158000438D41620385064B0649C362064B4363A4
:101590002C70FFF7D3FD2000F8BDC046FF7FFFFF92
:1015A0000000FFFF02800000FD190008036810B56D
:1015B00099691A68436B002B00D0984710BD70479B
:1015C0007047030070B500252022060042331D70CD
:1015D000013B1978040040361A7021290AD11123E1
:1015E000456303632039FFF7D9FD20003570FFF70D
:1015F000E6FF70BD1223456303630221FFF7CEFDB2
:1016000020003570FFF7DCFFF3E7704770470000FC
:101610000100036810B5040000201A684231087008
:101620000121500418D51A6818490A401A6023008D
:1016300041331A78292A15D1013A1A702123200042
:1016400023630121FFF7AAFD23000022403320007D
:101650001A70FFF7DAFF10BDD20B0A42E7D01A6802
:101660000B49E2E71A782A2AF5D1023A1A702223A6
:10167000200023630221FFF791FD23000022403365
:1016800020001A70FFF7C2FFE5E7C046FFBFFFFF6B
:10169000FF7FFFFF70470300F7B5282241331B7817
:1016A00004000168134093423CD1FE278D698E6986
:1016B0008B68CA68ED030192C268360CED0F3E409C
:1016C000022A25D19B059A0D5B0F5E403000062350
:1016D00018401E4210D1A36C0133A364A36C022BEB
:1016E00009D10633A064CB61230040331870290070
:1016F0002000FFF7CFFFF7BD802120000902FFF790
:101700004DFD2300002240331A70019A3A40EEE763
:1017100080210902FFF742FD2300002240331A70A6
:101720003200E4E70823CB61002340342370E2E772
:1017300070470000184B10B5C3620023020003631A
:101740000400202041321070537063634B0713D59F
:101750002368626A5B6A1370636A01336362238D74
:10176000002B09D0013B2385638D013B9BB2638530
:101770000423626C1343636420000849FFF70EFDE5
:10178000102223682000DA612300002240331A70FF
:10179000FFF7CEFF10BDC0460000FFFF0380000032
:1017A0007047704770470100020010B541310C7856
:1017B00000234032602C06D1403C0C700363137050
:1017C000FFF7F0FF10BD03631370FFF715F9F9E79A
:1017D00070B50200050004000020423241352B782C
:1017E0001070324A283BE2626085626C0A43626490
:1017F000022B2BD803212000FFF7D0FC28232B70CD
:101800002B4BA06B6363236B00282ED01A00102192
:10181000113A8A4329D123681A68520403D51A68F9
:1018200024490A401A6001F0D0F8012819D0A06BB1
:10183000214B00228363230040331A7001F0A0F88B
:10184000002811D0A06B836B98470DE020001B4946
:10185000FFF7A4FC2B78602B01D020232B700023F2
:10186000CFE72000FFF79FFF70BDE06B0028F8D0A6
:101870001022123B9343F4D123681A68120403D553
:101880001A680F490A401A6001F09FF80128E8D051
:10189000E06B094B00228363230040331A7001F090
:1018A0006FF80028E0D0E06BCDE7C0460000FFFFF6
:1018B000FD190008FFBFFFFF9F1E00080380000006
:1018C000FF7FFFFFF7B5036806001A6841360192F3
:1018D00020223578DA61082304000F009D43212D72
:1018E00050D140492000FFF759FC2563802223682E
:1018F0001202596820000A435A605A683A490A405D
:101900005A60FFF7F9FB019B01225B043ED5226878
:10191000364913680B401360A36B002B03D01B6880
:101920005B689BB263857B0711D504239F432368C3
:10193000626A5B6A1370636A01336362238D002BF2
:1019400005D0013B2385638D013B9BB26385638D8D
:10195000002B03D00423626C134363642300002232
:1019600042331A70656C626395421AD02000616C34
:10197000FFF72EFF3378282B03D139002000FFF723
:10198000D9FEF7BD222DB1D11949ABE7019BDB0B85
:101990001342C8D02268174913680B401360E36BE9
:1019A000BBE72700E36A144A403793420CD020007B
:1019B000FFF72EFE2023104A2000E26233702563D9
:1019C0003D70FFF7B5FEDCE720233278200033704E
:1019D00025633D70222A02D1FFF718FED1E7FFF7F9
:1019E00014FECEE70180000000E800FEFFBFFFFF0D
:1019F00002800000FF7FFFFF0000FFFF0300F7B53C
:101A0000403301931B780400C76A0E0015000220C2
:101A1000012B24D00123019A13704A091A4205D0E0
:101A20006A091A4202D02000FFF74CFF0123F20698
:101A300035D52A091A4232D0638D002B20D12300DC
:101A400041331A78282A0BD180229204974207D179
:101A500031002000FFF76EFE0020019B1870FEBDD4
:101A6000102219782368DA612929F5D12D498F428E
:101A7000F2D02000FFF740FB2000FFF7C9FDEBE7A5
:101A800010222368DA610423626C13436364264BDB
:101A90001F42E1D12000616CFFF79AFEDCE70123D1
:101AA00072071AD5AA081A4217D0638D002B0DD0E1
:101AB0002368626A5B6A1370636A01336362238D11
:101AC000013B2385638D013B9BB26385638D002BB6
:101AD000C2D1144B9F42BFD0CEE70123320706D5B7
:101AE000EA081A4203D02000FFF7D5FDB4E701232E
:101AF000B207B1D5DD401D42AED0638D002B0DD0B5
:101B0000636A22681978013391626362638D013BD5
:101B10009BB26385238D013B23859DE7024B1F42CA
:101B2000AAD099E70000FFFFFFFFFFFE73B5202258
:101B3000050003684135DA612B7804000E00212B83
:101B40002CD10121FFF72AFB1123236323682E499F
:101B50005A680A405A60002262632C4AE262F20626
:101B600005D51022DA61616C0C3A0A4362642A7866
:101B7000602A05D1720703D55B6ADBB20193019B32
:101B80002000FFF7B9FA636C2A78602A01D0002B95
:101B90000CD02000616CFFF71BFE73BD2B78222B4D
:101BA000D4D10221FFF7FAFA1223CEE72A78212AAC
:101BB00013D1013A2A7022002100236342321078A7
:101BC000403113700B70402803D12000FFF7E8FD6F
:101BD000E3E72000FFF7F3FCDFE72A78222ADCD1D5
:101BE000023A2A70220021002363423210784031E9
:101BF00013700B70402803D12000FFF7D2FDCCE713
:101C00002000FFF7DDFCC8E700E800FE0000FFFF52
:101C10000300F7B5403301931B780400C76A0E0038
:101C200015000220012B3CD00123019A13704A09B0
:101C30001A4205D06A091A4202D02000FFF742FE7C
:101C40000120F3065BD52B09034258D0AA0B1300E1
:101C5000ED0B2B4303424ED0E36B191E06D000213F
:101C6000054203D01B6859684B4259412300A06BC1
:101C70004133002805D0D20703D502685268002AF4
:101C800001D001291ED11A78282A0BD18022920472
:101C9000974207D131002000FFF74CFD0020019B47
:101CA0001870FEBD102219782368DA612929F5D150
:101CB00018498F42F2D02000FFF71EFA2000FFF7EC
:101CC000A7FCEBE710212268D1610422616C0A4372
:101CD00062641B78104ADBB21742DFD108229343BB
:101CE000212B01D1236301E0222BFBD02000616C6A
:101CF000FFF76EFDD2E710222368DA61CEE70123F9
:101D00003207CBD5ED081D42C8D02000FFF7C3FC39
:101D1000C4E7C0460000FFFFFFFFFFFE37B5050028
:101D200040352B7804000220012B17D0012308092D
:101D30002B70184213D01009184210D010222368BB
:101D40002000DA610423626C202113436364FFF7EF
:101D5000F5F92000FFF7D0F9002028703EBD0123DF
:101D6000080646D59009184243D0402123681A68D6
:101D70008A431A60628D002A2FD05968638D8905C5
:101D8000890DFF2B1BD9FF23238580235B040020B3
:101D9000228D0090D2B22000FFF7BCF9638D228D16
:101DA0009B1A9BB26385230041331A782368196814
:101DB000222A0FD1802212020A431A60CCE7638DD7
:101DC000E26A23851C4B9A4201D0E36ADFE7802355
:101DD0009B04DCE78022D201EEE75B689B0103D421
:101DE0002000FFF7EEFBB7E740212000FFF7F0FCF3
:101DF000B2E70123480613D59009184210D0638D2D
:101E0000002BF1D123685A689201A5D4E16A0A4AED
:101E10009142E5D180225968D2010A435A609BE77A
:101E20000123880600D497E752091A4200D193E7AC
:101E30002000FFF77BFE8FE70000FFFF036870B50F
:101E40009C6901211A68E50508D5D5090D4205D020
:101E5000456C2943416480214900D9610121650510
:101E600009D5D5090D4206D0456C07312943416497
:101E70008021C900D9610121A40509D5D2090A42EE
:101E800006D00222416C0A43426480229200DA6149
:101E90000B23416C194201D0FFF79AFC70BD806A98
:101EA00010B5836B002B01D000229A63C36B002B0B
:101EB00001D000229A63FFF776FC10BD4130007814
:101EC000C0B27047406C7047F0B5040041342278CE
:101ED00003000F000220D6B2202A18D11D00403581
:101EE0002A78012A13D0242222701B68233A196809
:101EF000074891431960196801400020196019686A
:101F00003943196019680A431A6026702870F0BDB9
:101F1000FFEFFFFF70B50500FA200D4B8000197828
:101F2000FEF706F90B4B01001868FEF701F900F007
:101F300085FD04000120002C09D1032D07D80238AB
:101F40002200290000F046FD2000034B1D6070BDFB
:101F5000100000200C000020140000204023084A3C
:101F600010B5116800200B431360FFF7D3FF041E68
:101F700003D1FEF7A9FE200010BD0124FBE7C046F7
:101F800000200240034A044B11681B785B18136061
:101F90007047C0461402002010000020014B186852
:101FA0007047C0461402002070B50400FFF7F6FF2A
:101FB0000500631C02D0044B1B78E418FFF7EEFF0A
:101FC000401BA042FAD370BD100000200C22194B18
:101FD00010B5D9680A40082A29D00C2A09D0042A49
:101FE0001DD11868144BC006C0171840134BC018F9
:101FF00010BD13488A02120F825C0902D868890F4B
:102000000131C00304D50F485043FEF791F8EFE7C4
:102010001B68DB0601D50C48F6E70848F4E780208A
:102020005B6800021B045B0F01339840E0E7054842
:10203000DEE7C0460010024000E548FF0024F4003F
:10204000163E000800127A0000093D00F0B50500B8
:1020500087B0002854D00C23C04C0268E668E768BB
:102060001E4080235B021F40D2073DD42B689B0794
:1020700000D586E02B68DB0628D5002E00D0DEE0F8
:1020800023689B0502D5AB69002B39D06268B4493F
:102090002B6A0A401A4362606168EA690902090A08
:1020A00012060A43626080225B0B013312029A40DF
:1020B0001300E16800200A06AA49120F8A5CD34087
:1020C000A94A1360FFF726FF002830D12B681B07B1
:1020D00000D5EBE02B685B0700D50DE16B6A002BA8
:1020E00000D092E1002022E0082E03D00C2E09D16E
:1020F000002F07D023689B03B8D56B68002BB5D1A0
:10210000012014E06A689A4213D1226813432360C5
:10211000FFF744FF01908022236892021342A5D169
:10212000FFF73CFF019BC01A6428F4D9032007B0D5
:10213000F0BDA021C9028A4205D180222168D202C5
:102140000A432260E1E72168884801402160216854
:102150000B400593059B864923680B402360002AAA
:10216000D6D1FFF71BFF0190802223689202134211
:1021700000D17BE7FFF712FF019BC01A6428F3D957
:10218000D4E72022EB68134203D021689343114324
:102190002160042E03D00C2E23D1002F21D12268E0
:1021A000520701D5002BABD061682A697148120231
:1021B00001400A430921626022688A431343236075
:1021C000FFF704FFE368674A1B061B0FD35CD84088
:1021D000654B18600020FFF79DFE002800D149E7FD
:1021E000A5E7002B19D0092122688A4313432360F5
:1021F000FFF7D4FE070004222368134207D0626869
:102200002B695C491B020A401343636032E7FFF706
:10221000C5FEC01B0228EED988E70122236893433C
:102220002360FFF7BBFE070004222368134200D19E
:1022300020E7FFF7B3FEC01B0228F5D976E7AB69AC
:10224000002B20D0802322685B0013432360FFF71C
:10225000A5FE070080222368920013420DD0636818
:102260003F4A13402A6A134363606268EB691202B3
:102270001B06120A1343636028E7FFF78FFEC01B9B
:102280000228E7D952E723683B4A13402360FFF74F
:1022900085FE0700802223689200134200D115E7D3
:1022A000FFF77CFEC01B0228F4D93FE76A690123CF
:1022B000002A10D0226D13432365FFF76FFE07003D
:1022C0000222236D134200D004E7FFF767FEC01B14
:1022D0000228F5D92AE7226D9A432265FFF75EFEB0
:1022E00007000222236D134200D1F3E6FFF756FEEA
:1022F000C01B0228F5D919E780230021A26B5B05DA
:1023000001911A4204D1A26B1343A36301230193E9
:1023100080221A4F52003B68134208D08022AB68DB
:10232000520093422CD1226D134323654DE080224D
:102330003B68520013433B60FFF730FE80235B0095
:10234000029003933B68039A1342E7D1FFF726FEFE
:10235000029BC01A6428F5D9E8E6C0460010024086
:10236000FF1FFFFFFE3D00080C000020FFFFFEFFE7
:10237000FFFFFBFFFFE0FFFFFFFEFFFF00700040DD
:10238000002B16D1236D514A13402365236D504A0B
:1023900013402365FFF702FE07008022236D9200A1
:1023A00013421AD0FFF7FAFD4A4BC01B9842F4D9EA
:1023B000BCE6A021C9008B4218D18023216DDB002F
:1023C0000B432365236D1A432265FFF7E7FD0700E2
:1023D0008022236D9200134210D0019B012B00D06C
:1023E0007CE6A36B3C4A1340A36377E6236D374A30
:1023F00013402365236D364A134096E7FFF7CEFD61
:10240000344BC01B9842E3D990E60C2E43D0334A9C
:10241000022B2ED12368802713402360FFF7BEFDD7
:102420000600BF0423683B421DD1E96AAB6AE2683B
:102430000B432B4980260A4013432A6BB6041343EF
:10244000E360802322685B0413432360FFF7A6FD4B
:1024500005002368334200D044E6FFF79FFD401B90
:102460000228F6D962E6FFF799FD801B0228D9D928
:102470005CE62368802613402360FFF78FFD05008C
:10248000B6042368334200D12CE6FFF787FD401BDA
:102490000228F6D94AE61800012B00D147E680222F
:1024A000E368A96A52021A408A4200D028E6F02264
:1024B000E96A92031A408A4200D021E6C02212043F
:1024C00013402A6B934200D10CE619E6FFFEFFFF92
:1024D000FFFBFFFF88130000FFFFFFEFFFFFFFFE82
:1024E000FFFF02FFF7B5041E019101D10120FEBDDF
:1024F0000122514D01992B6813408B4227D322684A
:1025000093072FD4D30735D401232A6801991A40A1
:102510008A4200D981E02268484D530700D584E003
:10252000130706D5EA6823694549DB000A401343CF
:10253000EB60FFF74BFDEB68424A1B061B0FD35CB9
:10254000D840414B18600020FFF7E4FCCFE72B6830
:10255000019993430B432B602B681340019A9342DC
:10256000C4D1CCE7F0203549CB688343A06803434E
:10257000CB60C7E7314E62683368022A19D19B03EA
:10258000B4D50321F3688B431343F360FFF706FDD3
:1025900063680700022B19D10C22F3681340082B43
:1025A000B2D0FFF7FBFC294BC01B9842F4D90320A3
:1025B0009DE7032A02D19B01E3D497E7012A02D1C8
:1025C0005B07DED492E79B05DBD48FE7032B0BD1AF
:1025D0000C22F3681340934296D0FFF7DFFC1B4BAD
:1025E000C01B9842F4D9E2E7012B10D00C22F3680B
:1025F000134289D0FFF7D2FC144BC01B9842F5D987
:10260000D5E7FFF7CBFC114BC01B9842CFD80C226B
:10261000F3681340042BF4D176E72A689A432A60C2
:102620002A681A4200D176E760E7EB6808490B4058
:10263000E1680B43EB6073E70020024000100240AA
:10264000FFC7FFFFFE3D00080C00002088130000BC
:10265000FFF8FFFF014B18687047C0460C000020D0
:10266000044B054ADB685B055B0FD35C034A1068CB
:10267000D8407047001002400E3E00080C000020B9
:10268000044B054ADB689B045B0FD35C034A10686C
:10269000D8407047001002400E3E00080C00002099
:1026A0000368F7B505009B063DD580230021504CFB
:1026B0005B05A26B00911A4204D1A26B1343A36382
:1026C0000123009380274B4E7F0033683B4251D05B
:1026D0006B68C022C0201E00216892028003170090
:1026E0001640034001408B4255D1236D1A003A40F9
:1026F0003B4257D16968C0230A009B021A409A42A4
:1027000007D123683C480340C020800301400B43AD
:102710002360236D1A43009B2265012B03D1A36B19
:10272000364A1340A3632A68930706D50C20304924
:10273000CB6C8343A8680343CB64530706D52C496D
:102740002F48CB6C0340E8680343CB64130706D5DE
:1027500027492C48CB6C034028690343CB640020F5
:10276000130617D5224A2849D36C0B4069690B43DD
:10277000D3640FE033683B433360FFF70FFC0190F5
:1027800033683B42A4D1FFF709FC019BC01A6428BF
:10279000F6D90320FEBD9642A7D1236801209B03F2
:1027A000A3D5F7E7B242A5D02B689B06A2D580221D
:1027B000216D206D120302432265226D134B1448D4
:1027C0000B40024022652365CB0500D492E7FFF75A
:1027D000E5FB80270600BF00236D3B4200D089E760
:1027E000FFF7DCFB0B4B801B9842F5D9D1E7C046C5
:1027F0000010024000700040FFFFCFFFFFFFFFEF1F
:10280000FFF3FFFFFFCFFFFFFFFFF3FFFFFFFCFF23
:10281000FFFFF7FF881300000023F0B585B00A68BA
:102820001400DC4001D105B0F0BD012415009C402E
:1028300025400295224200D189E010254A685E00B9
:102840000192AA430D3DB5409446013AED43012A59
:102850000FD8CA688768B2402F403A430127826088
:102860004268A2431400019A12093A409A40224356
:1028700042608A68C468B2402C402243C26062460B
:10288000022A0FD1DA08072492008218176A0392ED
:102890000F221C40A400A24097430A69A24017439C
:1028A000039A1762032402681540019A2240B2403D
:1028B00080241543019A64050560224247D0012512
:1028C0000F27244C626B2A4302351D40AD00AF40F8
:1028D0006263214A9C08A400A418A6680022BE4393
:1028E000A027FF05B84208D01C4F0132B84204D0DF
:1028F0001B4F0132B84200D00432AA403243A260DA
:10290000184A029C1668029D019FE4433543FF0369
:1029100001D43500254015605668029D019F35435E
:10292000BF0301D43500254055609668029D019F84
:102930003543FF0201D4350025409560D568029EDD
:10294000019F2E43BF0201D425402E00D6600133E3
:1029500065E7C0460010024000000140000400503E
:10296000000800500004014000690840411E8841F1
:10297000C0B27047002A01D0816170478162FCE7D4
:1029800070B5841DE37F022B04D00423C363033B93
:10299000180070BD0E210368456C1A688A431A60DE
:1029A00001221968914319601C232B4015009D409A
:1029B000016C431D4D60E2770024DC77826B1300CD
:1029C000A242E5D090472300E2E70630C07FC0B2C4
:1029D0007047000030B5FF2503242A000440E400BE
:1029E000A24089012940D243A140C3B200280BDA9A
:1029F0000F200340083B0A489B089B001B18D8691E
:102A000002401143D96130BD064B80088000C018D8
:102A1000C0239B00C45822401143C150F3E7C04675
:102A200000ED00E000E100E01F2318401E3B834062
:102A3000014A13607047C04600E100E08022431E57
:102A40005204012093420DD2C021074A0748536027
:102A5000036A09061B021B0A0B43036200200723BB
:102A6000906013607047C04610E000E000ED00E0A9
:102A7000802210B50368D205904202D00D4CA042CE
:102A80000CD17024A3434C682343904202D0094ADE
:102A9000904203D1084A1340CA68134380229343EB
:102AA0000A69134303608B68C3620B688362012366
:102AB000436110BD00080140FFFCFFFF012230B55B
:102AC0007325036A93430362036A44688269AA43D5
:102AD0000D682A430225AB438D68446082614A68D1
:102AE0002B434263036230BD1022036A30B5934327
:102AF0000362036A094C4568826914400A6812023D
:102B000022432024A3431C008B6845601B01826183
:102B10004A6823438263036230BDC046FF8CFFFFD7
:102B20001F2310B5012419408C408A40036AA34337
:102B30000362036A1A43026210BD70B504000120EB
:102B4000002C14D0250039352B78DAB2002B05D1B2
:102B50002300383320001A70FDF7ACFF02232B70DE
:102B60002068211DFFF784FF012300202B7070BD1A
:102B70000100022339310B70036807209A68024074
:102B8000062A03D00122186802431A60012300209C
:102B90000B707047704770B504000120002C14D0F2
:102BA000250039352B78DAB2002B05D123003833D4
:102BB00020001A70FFF7EEFF02232B702068211D02
:102BC000FFF756FF012300202B7070BD10B50400E5
:102BD00001220068FFF7A4FF072123689A680A40D2
:102BE000062A03D0012219680A431A60002010BD8A
:102BF000F8B5040002263834257803003000012D92
:102C00000FD01D000138393520702E70082A2AD0C7
:102C100008D8002A1FD0042A21D0012300202B70BD
:102C20002070F8BD0C2AF8D11B681A481A6A1A4E8F
:102C300002401A621A6A5F68D86930400E6836022C
:102C40003043164E16408A68496812035F6032436B
:102C5000D86119641CE01868FFF730FFDDE71868D9
:102C6000FFF742FFD9E773261B680D481A6A024036
:102C70001A621A6A5F68D869B0430E683043094E19
:102C800016408A68496812025F603243D861D9638E
:102C90001A62C2E7FFEFFFFFFF8CFFFFFFDFFFFFBE
:102CA000FFFEFFFFFFFDFFFFF0B5040002223834F6
:102CB000257803001000012D24D01D000126393590
:102CC00026702A701B6845489A6802409A600A6814
:102CD000602A55D02FD8402A00D169E013D8202A85
:102CE00004D009D810211000884307D170209968BA
:102CF00081430A43072140E0302AF7D00123002016
:102D00002B702070F0BD502AF8D14868CA68196A43
:102D10001F6A1201B7431F62F0279E69BE43324308
:102D20000A26B14301439A61196270219A688A4365
:102D30001100572221E0702A12D0802080018242A7
:102D4000DCD19A6826484E6810408A68C9683243C8
:102D500009020A4302439A6080229968D2010CE07A
:102D60009A681F484E6810408A68C9683243090251
:102D70000A4302439A60772299680A439A60BDE742
:102D80001026186A4A68B043C96818629E69154FD0
:102D900009033E403143A026186A99617021B0436F
:102DA000120102431A629A688A4311006722E4E71B
:102DB0004868CA68196A1F6A1201B7431F62F02780
:102DC0009E69BE4332430A26B14301439A611962A8
:102DD00070219A688A4311004722CEE78800FFFFDE
:102DE000FF00FFFFFF0FFFFF70B504000222383421
:102DF000257803001000012D13D0180070263930FB
:102E000002701D686A68AB68B2430E684968324355
:102E10008026B3430B436A60AB600123037000203C
:102E2000207070BDF8B505002C69AA6803682243BC
:102E30006C69C169224318687E4C0A4320400243F2
:102E40001A605A687C487D4C0240E86802435A6028
:102E5000A869A34201D02A6A10439A68784E32408A
:102E600002439A60774A934215D10C20764BDA6C74
:102E700002407648845C80221202914200D095E0A4
:102E8000082C00D98FE02000FDF748F9526B738DB4
:102E9000858D8D8D8800A34200D0C4E0C0218020A4
:102EA000694A0901D36C00010B40834217D007D84F
:102EB000002B0AD08022D200934236D0012409E0B0
:102EC0008B42FBD18020000213E0FFF7C9FB0024F6
:102ED000A0420ED1002320002B666B66F8BD1023A4
:102EE0001068184043425841594B40421840594BD2
:102EF000C01803236A6853438342DFD81303834215
:102F0000DCD300275608040E03029B197C411800ED
:102F100021003B00FDF798F94F4BC2184F4B9A42E6
:102F2000CCD82B683C00D860D4E7FFF74FF8CEE749
:102F3000FFF796FB6B6840005B086968C018FDF7F7
:102F4000F7F880B20300464A103B9342B6D80F23ED
:102F500002009A43130000072A68400F1843D0600C
:102F6000B8E7FFF78DFB6B6840005B086968C01825
:102F700009E01A681023140069681C4048081A42C6
:102F800006D0384BC018FDF7D3F8002480B2D9E73B
:102F9000354BC018D3E7FFF719F8E4E76B6858081A
:102FA00080235B02E2E701240020CBE7082C3ED817
:102FB0002000FDF7B3F8050F163C303C3C3C3300D5
:102FC000FFF74EFB6B6869685B081818FDF7B0F8EF
:102FD00080B214E0FFF754FB6B685B086968C018A7
:102FE00009E01A681023140069681C4048081A4256
:102FF0000ED0184BC018FDF79BF8002480B20300D8
:10300000174A103B934200D958E72B68D86061E714
:10301000164BC018DAE7FEF7D9FFDDE76B685808F2
:1030200080231B02DAE780231B029942BBD00124D4
:103030000020E4E7F369FFEFFFCFFFFF0048004007
:10304000FFF4FFFF00440040001002401F3E000854
:10305000001BB70000093D0000FDFFFFFFFC0F0053
:10306000EFFF000000127A000048E8010024F4009D
:10307000436A30B5DA0706D50168284C4A68224011
:10308000846A22434A609A0706D50168244C4A683C
:103090002240C46A22434A605A0706D50168214C7F
:1030A0004A682240046B22434A601A0706D5016829
:1030B0001D4C4A682240446B22434A60DA0606D51A
:1030C00001681A4C8A682240846B22438A609A06FF
:1030D00006D50168164C8A682240C46B22438A6078
:1030E0005A0610D50168134D4A68046C2A402243E1
:1030F0004A6080225203944205D14A680E4C224015
:10310000446C22434A601B0606D502680B4953688B
:103110000B40816C0B43536030BDC046FFFFFDFF89
:10312000FFFFFEFFFFFFFBFFFF7FFFFFFFEFFFFF44
:10313000FFDFFFFFFFFFEFFFFFFF9FFFFFFFF7FF37
:10314000F8B504000D0017001E002268D3692B405B
:103150005B1B59424B41BB4201D000201BE0069B48
:103160000133F3D0FEF71AFF069B801B984201D86B
:10317000002BEAD1236808491A6803200A401A6024
:103180009A68A331FF318A439A6020236367A3675B
:10319000002370342370F8BD5FFEFFFFF0B585B0EB
:1031A0000393436F04000D0016000220202B4DD125
:1031B000013800294AD0002A48D08023A2685B0148
:1031C0009A4204D12369002B01D101423ED1230050
:1031D00070331A780220012A38D001221A70002395
:1031E000E36721336367FEF7D9FE230050331E8067
:1031F00002331E8002938023A268070000265B0131
:103200009A4204D12369B34201D12E001D0023004C
:1032100052331B889AB2002B0DD1039B402100939F
:1032200020003B00FFF78CFF00280ED120237034D4
:10323000636020700AE0039B0022009380213B0022
:103240002000FFF77DFF002802D0032005B0F0BD6D
:103250002268002D0BD133880236DB05DB0D93622B
:10326000029B029A1B88013B9BB21380CFE72B780D
:1032700001359362F4E7000073B500260400C667C9
:10328000FEF78CFE236805001B681B0715D4236816
:103290001B685B070AD580210E4B0022009320009B
:1032A0002B00C903FFF74CFF002811D12023002079
:1032B0006367A367703420700BE08021054B3200F8
:1032C0000093890303002000FFF73AFF0028DED0B7
:1032D000032076BDFFFFFF0110B5041E01D10120C0
:1032E00010BD436F002B04D1020070321370FDF744
:1032F00093FC2423012122686367136820008B4319
:103300001360FFF78FFD0128E9D0636A002B02D01C
:103310002000FFF7ADFE236807495A6820000A40E5
:103320002A215A609A688A439A60012219680A43DE
:103330001A60FFF7A1FFD3E7FFB7FFFF084B13B5F4
:10334000040008491868FCF7F3FE44430194019B0C
:10335000002B00D113BD019B013B0193F7E7C04651
:103360000C00002040420F000321036870B59A68EA
:1033700004000A40012A04D11968114201D000203A
:1033800070BD9968134A114208D010230120626D64
:1033900013436365A36D0343A365F1E701259A68B1
:1033A00028002A439A60FFF7C9FFFEF7F7FD0600E1
:1033B00023681B682B42E2D1FEF7F0FD801B0A2830
:1033C000F6D91023626D012013436365A36D1D437D
:1033D000A565D5E71700008070B504000120002C1A
:1033E0001BD0636D002B06D122005032A365200054
:1033F0001370FDF7D7FC636DDB0606D42368042247
:10340000996808001040114208D01023626D012015
:103410001343636500235034237070BD626D5549BA
:10342000114002220A436265032299681140524A00
:10343000012902D11D680D4219D180266168F60567
:103440004D006D08B54203D080252D06A94276D1E6
:103450001D69AD00AD081D611D692943196118255D
:10346000D968A943D960D968A5682943D96011688A
:10347000424D29401160616B15684906294311606E
:10348000802299685205114202D199680A439A60D4
:10349000DA683B490A402169DA60DD68E26802299E
:1034A00000D10420266B611C32432A43A569C97FE1
:1034B000AD032A43E569ED032A434D032A43250062
:1034C0002C352D786D002A430243C220DA60626AEF
:1034D000FF30824204D0A56AD8682A430243DA60EA
:1034E000A21CD27F012A06D1002934D18022D968BA
:1034F00052020A43DA60E16B1A69012933D121488B
:10350000656C02401A61226C18692A43A56C2A4333
:1035100002431A611A691143196107215A6900208F
:103520008A435A615A69A16B0A435A610322A06512
:10353000636D93431A000123134363656DE71D69AF
:10354000114EAD00AD081D61156835401560156858
:103550002943116083E72021606D01436165A16DFE
:103560000A43A265C7E701210A42D6D01A698A43F5
:103570001A61D2E7FDFEFFFF08270140FFFFFFFDB4
:103580001902FEFF03FCFFFFFFFFC3FF036870B5D6
:103590009B68040002205B071AD4250050352B7865
:1035A000012B15D001232B70E369012B11D1636D21
:1035B0000B4A00201A4080235B0013431C226365E2
:1035C000A065287023681A609968183A0A439A60BF
:1035D00070BD2000FFF7C8FE0028E8D0F8E7C0461D
:1035E000FEF0FFFFF8B5466904000D00082E0DD06F
:1035F00003680120DB680C26034207D02023626D9C
:1036000050341343636000232370F8BDFEF7C6FCFB
:10361000070023681A68164224D08022616D920048
:103620000A436265C022D9681201114213D1621C9B
:10363000D27F002A0FD11A6812070CD59A68520758
:1036400023D40C215A688A435A60626D1349114091
:1036500001220A4362650020A2698242D5D10C2270
:103660001A60D2E76A1CD5D0002D08D10423626D00
:10367000503413436360002303202370C5E7FEF733
:103680008DFCC01BA842C4D9F0E72022616D0A431B
:1036900062650122A16D0A43A265DCE7FEFEFFFF21
:1036A0000368186C70470000F8B5040050342278A5
:1036B00003000D000220012A0BD0013820701A6887
:1036C0009168490706D52022596D0A435A6500239F
:1036D0002370F8BD80232868194E6F684103DB0210
:1036E000490B0340B74219D0906A01439162002B05
:1036F00008D08023134A1B0411680A200B4313606F
:10370000FFF71CFE2B689B0305D580230D4ADB03C6
:1037100011680B43136000202070DAE7956A8D432F
:103720009562002B04D0074A074913680B401360C9
:103730008303F0D5034A054913680B40EAE7C04606
:103740000110000008270140FFFF7FFFFFFFBFFFC0
:10375000F8B5050050352B7804000220012B44D029
:10376000012303222B70236898681040012809D197
:103770001A68024206D02023626D1343636500235A
:103780002B7032E0626D1949114002220A43032175
:103790006265DE68DA688A43DA6080229968120618
:1037A0000A439A60FEF7FAFB070023689A68002A2A
:1037B0000CDB0322D96816400E43DE60636D0020E7
:1037C00093431A00012313436365D8E7FEF7E6FB32
:1037D000C01B0A28E9D91222636D012093431A0005
:1037E00010231343636500232B70F8BDFDFEFFFF1C
:1037F0000CB4F0B587B00CAE08CE1A4D03931A4B3B
:103800001A4A5B5C00903F21280000F0E1F9C343B5
:103810000400DB17FF271C4040232740039AD91BD5
:10382000E8193300059600F0B9F9C2B20300101E82
:1038300013D0FF210B40DB19BF393F2B01DC1419DA
:10384000E1B20D230A226B544B1C02312800DBB27B
:10385000C9B2EA54FDF720FA012007B0F0BC08BC59
:1038600002B018476D000020353E00082C3E0008CD
:10387000F0B505000E0001240B6985B0CF680193F7
:1038800021002800FCF754FCB84206D20027002C87
:1038900005D1019B1C7005B0F0BD7C43F0E728000A
:1038A0002100FCF7CBFCF3680D000290190020000A
:1038B0000393FCF73DFC002F07D1029B002B04DC97
:1038C000039BA34214D80400E1E7029A3023092A9B
:1038D00005DD0421327807330A4200D12033029AF1
:1038E00001379B18019A1370130001330193EAE723
:1038F0003023F4E7F7B50600150054681369019109
:103900001B1962429A5C002A01D0002C38DC2B7A09
:103910005A1E93412A78E41A930703D5EB68102BBB
:1039200030D1023C092327001A4235D0297A0029D8
:1039300002D03000019B98472B789B070ED5EB688F
:10394000102B31D13021019B300098472B78582122
:103950005B0700D420313000019B98472B7827006B
:10396000DB072AD42F6901377B1E197800292CD157
:1039700009222B781340082B01D1002C29DCF7BD3C
:10398000013CBEE7083B59424B41E41ACAE72021FB
:103990003000019B9847013F002FF8DCE343DB1721
:1039A000621E1C40141BC1E7082BD7D13021D2E77F
:1039B00030213000019B9847013F002FF8DCE343A2
:1039C000DB17621E1C40141BCCE73000019B98479C
:1039D000C9E720213000019B9847013CCDE783686F
:1039E0000268934201D24268D154836801338360F4
:1039F0007047F0B505000E008BB01C0002AB0993B8
:103A00001178531C0093002901D10BB0F0BD25297A
:103A100002D02800B04775E000230B2005AA1178DA
:103A200006938143180011700099137201934A1C88
:103A3000097894460092002904D1002810D005AFDF
:103A40003A780AE02D2921D0302922D0232923D009
:103A5000002805D005AF38780200082010433870E0
:103A6000019A002A04D0012705AA10783843107063
:103A7000002B04D0022305AA1078034313700B0017
:103A8000303B092B23D800220A200DE0012061469B
:103A9000CDE701220192FAE70123F8E742439A18A1
:103AA0006346197801239C44634600930B00303B26
:103AB000DFB2092FF2D9313B052B03D80A330A2B89
:103AC000ECD003E00B00413B052BF7D906922E29E1
:103AD0000DD105AA13782D390B43137063461A00D4
:103AE000117801330A00303A0093092AF7D969297D
:103AF0000ED01FD858292ED006D8002900D184E72F
:103B0000252986D0009A7BE7632939D06429F9D129
:103B10000A2301CC05AFFB60002802DA23334042C0
:103B20003B723900FFF7A4FE3A0031002800FFF78E
:103B3000E1FEE7E708006F38C3B2092BE2D8092895
:103B4000E0D8FCF7E1FA1BDFDFDF20DF05DFDF086D
:103B50000A2308930CE01023583908934B4259412B
:103B600002AA8B00117B04229143194302AB197303
:103B700001CC05A9FFF77CFE05AAD6E70823E8E7F4
:103B800002CCC9B245E708CC3100280005AA099348
:103B9000FFF7B0FE02AB0993B4E700001FB50024A5
:103BA000A1420ED001390290019101A80749039466
:103BB000FFF71FFF0399019B029A994204D25454C4
:103BC000039C200004B010BDD454F9E7DF3900088D
:103BD0000CB407B504AB04CB0193FFF7DFFF03B0D0
:103BE00008BC02B01847000010B5029C002805D0A0
:103BF000002A03D0002B01D0002C06D104210D4A4D
:103C00000D48FFF7F5FD002010BD0329FBD9017811
:103C1000117041781970C17821701278013A032A25
:103C2000F1D8002002221B78013BDBB29A424041CE
:103C3000C0B2E9E73C3E0008533E00081348854601
:103C400013480168090E134A914205D112481349DD
:103C50000160134813490160002103E0124B5B58D7
:103C6000435004311148124B42189A42F6D3114A7C
:103C700002E00023136004320F4B9A42F9D3FDF7A0
:103C800031F800F01DF8FCF7F5FBFEE70008002016
:103C9000040000001F00000034100240010000007A
:103CA0000000014000000000683E00080000002005
:103CB000180000201800002018020020FEE7000075
:103CC00070B500260C4D0D4C641BA410A64209D102
:103CD000002600F02BF80A4D0A4C641BA410A642E3
:103CE00005D170BDB300EB5898470136EEE7B3003D
:103CF000EB5898470136F2E7603E0008603E000846
:103D0000603E0008643E0008002310B59A4200D1CE
:103D100010BDCC5CC4540133F8E703008218934211
:103D200000D1704719700133F9E70000F8B5C046BB
:103D3000F8BC08BC9E467047F8B5C046F8BC08BC45
:043D40009E467047E4
:103D4400000000506C616E7453656E736F72207660
:103D5400302E31004D41494E0041707220313320E4
:103D640032303231004275696C6420646174653AA2
:103D74002025732025730030313A30333A3239002C
:103D84005375636365737300490054004D0041002B
:103D9400440046460054582074696D656F7574007C
:103DA400543A25642E256443202D204D3A20256461
:103DB400202D204C3A2025640053454E5300496E73
:103DC40076616C696420617267756D656E7421003B
:103DD40049324300496E76616C696420706F696E84
:103DE40074657221006E54584275666665724C653E
:103DF4006E20746F6F20626967000000000000008D
:103E04000000010203040607080900000000010283
:103E14000304030406080C101820300010101004CA
:103E240010101002101010085B25635D5B25735D94
:103E3400005444495745464F496E76616C69642085
:103E440063616C6C20617267756D656E74210050DE
:043E54005300000017
:083E580030C4FF7F01000000EF
:043E6000E90000086D
:043E6400C100000891
:103E6800FF0000000000000000000000000020002B
:083E780001000000040000003D
:0400000508003C3D76
:00000001FF
